:03F0000002F00813
:03F0610002F003B7
:05F0030012F7AA80FED7
:04F06400AA82AB834E
:05F068001ABAFF011BB4
:0EF06D00C3E49A74808BF063F08095F0500F2E
:04F07B007CB07D04E4
:05F07F001CBCFF011D97
:06F08400EC4D70F780DE88
:01F08A002263
:0EF08B0090DF077412F090DF08E4F090DF17BA
:0EF09900E044C0F090DF1C74EAF090DF1D74BC
:0EF0A7002AF090DF1EE4F090DF1F741FF0903F
:0EF0B500DF237488F090DF247431F090DF25A3
:09F0C3007409F090DF14E4F0225E
:07F0CC007401B52602800764
:07F0D3007402B5261080074E
:07F0DA0090DF0C74ECF02242
:07F0E10090DF0C740CF0221B
:07F0E80090DF0C746CF022B4
:0EF0EF00AA82AB83ACF0FDC002C003C004C017
:0EF0FD000512F9ADAE82AF83A8F0F9C006C0CF
:0EF10B0007C000C0019030E975F025743B127A
:0EF11900F8B3AE82AF83A8F0F9E58124FCF5CF
:0EF12700818E828F8388F0E912F9C0AE82AF2C
:0EF1350083A8F0D005D004D003D00290DF09EB
:0EF14300E8F090DF0AEFF07F0078007900908E
:0CF15100DF0BEEF0E525700FC3EA9480A0
:0BF15D00EB944BEC94F4ED9412402274
:0CF168007401B5250CC3EB94BAEC94457F
:05F17400ED94194011AB
:0CF179007402B52513C3EB9474EC948B66
:05F18500ED943250077B
:07F18A0090DF1D740AF02262
:07F1910090DF1D742AF0223B
:0DF1980012F0EF75E10175E1029000021226
:0CF1A500F064E52A75F008A4FAABF0EA6B
:0AF1B1002400FCEB3400FD90DF09A0
:0CF1BB00E08C828D83F0EA2400FAEB3433
:0CF1C70000FB74012AFCE43BFD90DF0A11
:0EF1D300E08C828D83F074022AFCE43BFD90F8
:0EF1E100DF0BE08C828D83F074032AFCE43B8C
:0EF1EF00FD90DF1CE08C828D83F074042AFCFE
:0EF1FD00E43BFD90DF1DE08C828D83F07405F5
:0EF20B002AFCE43BFD90DF1EE08C828D83F038
:0EF2190074062AFCE43BFD90DF3AE0FE63063B
:0EF22700808C828D83EEF074072AF582E43B22
:08F23500F583E4F075E1042209
:09F23D0085822B85832C7401B538
:04F246002602800715
:07F24A007402B52650801488
:07F25100753A03753B0175DE
:06F258002E44752FC37562
:07F25E003000753100806FE4
:07F26500753A2A753B147590
:06F26C002E88752F2B75A2
:08F27200300A753100740A2511
:09F27A002BF582E4352CF58375B7
:06F283000814E4F5091275
:07F28900F88A8582088583E5
:09F290000990001412F9F98582BD
:06F299002B85832C80355B
:07F29F00753A0D753B057582
:06F2A6002E10752F0D75FE
:06F2AC00300375310085FE
:08F2B2002B82852C83A3A375B8
:06F2BA000805E4F509124D
:07F2C000F88A8582088583AE
:09F2C7000990000512F9F9858295
:04F2D0002B85832CDB
:0AF2D400C37467952B7402952C405B
:04F2DE000302F4240F
:0AF2E200752D02AC3A7D0074C2C322
:0CF2EC009CFE74039DFFE53BC313F87902
:0CF2F800002EF582E93FF583AE3B7F005D
:0AF304008E088F09C004C005C00682
:0EF30E00C007C000C00112FAD3AA82AB83D0A0
:0AF31C0001D000D007D0068E088F44
:0CF32600098A828B83C006C007C000C0AB
:09F332000112F9F985823C858382
:0CF33B003DD001D000D007D006D005D096
:0CF347000474ED2CF58274023DF5838EF9
:0AF35300088F09C004C005C006C001
:0EF35D0007C000C00112FAD3AA82AB83D00110
:0AF36B00D000D007D0068E088F09ED
:0DF375008A828B83C006C007C000C0011251
:07F38200F9F985823E858345
:0CF389003FD001D000D007D006D005D046
:0CF395000474192CF58274013DF5838E80
:0AF3A100088F09C004C005C006C0B3
:0EF3AB0007C000C00112FAD3AA82AB83D001C2
:0AF3B900D000D007D0068E088F099F
:0DF3C3008A828B83C006C007C000C0011203
:0EF3D000F9F9AA82AB83D001D000D007D00695
:0EF3DE00D005D00474E1C39CFC74019DFDE8D1
:0AF3EC002CF582E93DF5838E088FB1
:0CF3F60009C002C003C006C00712FAD311
:0BF40200AC82AD83D007D0068E088FCF
:0CF40D00098C828D8312F9F9AC82AD836A
:0BF41900D003D0027E007F0102F5C38B
:0AF42400C37471952B7401952C4000
:04F42E000302F4FCE5
:05F43200752D01853A73
:08F437004075410074E1C3952A
:06F43F0040F54274019546
:04F4450041F543E565
:07F449003BC313F888447572
:05F450004500E5442524
:06F4550042F582E5453599
:05F45B0043F583853B31
:05F46000427543008528
:03F46500420885D5
:03F4680043091243
:04F46B00FAD3854209
:03F46F00088543CA
:06F472000912F9F9858280
:07F478003C85833D747A25F9
:0AF47F0040F58274013541F58385E4
:03F48900420885B1
:03F48C004309121F
:04F48F00FAD38542E5
:03F49300088543A6
:06F496000912F9F985825C
:07F49C003E85833F74ED255E
:0AF4A30040F58274023541F58385BF
:03F4AD004208858D
:03F4B000430912FB
:04F4B300FAD38542C1
:03F4B70008854382
:0CF4BA000912F9F9AA82AB837469C395AA
:08F4C60040F874019541F9E5DD
:0AF4CE004428F582E54539F58385F1
:03F4D80042088562
:07F4DB004309C002C0031247
:04F4E200FAD3854292
:03F4E60008854353
:0CF4E9000912F9F9AC82AD83D003D00207
:07F4F5007E027F0002F5C357
:05F4FC00752D00853AAA
:08F50100447545007469C395CF
:06F5090044F54274019577
:04F50F0045F543E596
:07F513003BC313F8884075AB
:05F51A004100E5402561
:06F51F0042F582E54135D2
:05F5250043F583853B66
:05F52A0042754300855D
:03F52F004208850A
:03F5320043091278
:04F53500FAD385423E
:03F53900088543FF
:06F53C000912F9F98582B5
:07F542003C85833D7419258F
:0AF5490044F58274013545F5838511
:03F55300420885E6
:03F5560043091254
:04F55900FAD385421A
:03F55D00088543DB
:06F560000912F9F9858291
:07F566003E85833F747A2506
:0AF56D0044F58274013545F58385ED
:03F57700420885C2
:03F57A0043091230
:04F57D00FAD38542F6
:03F58100088543B7
:0CF584000912F9F9AA82AB8374C2C39586
:08F5900044F874039545F9E508
:0AF598004028F582E54139F583852E
:03F5A20042088597
:07F5A5004309C002C003127C
:04F5AC00FAD38542C7
:03F5B00008854388
:0CF5B3000912F9F9AC82AD83D003D0023C
:04F5BF007E017F0248
:06F5C300C3E53C952BE5B9
:06F5C9003D952C50138556
:03F5CF003C2B854D
:03F5D2003D2CE5E8
:05F5D50025B52D248E78
:04F5DA002D8A2B8BC0
:03F5DE002C801C62
:06F5E100C3E52B953EE599
:06F5E7002C953F50118538
:03F5ED003E2B852D
:03F5F0003F2CE5C8
:05F5F30025B52D068F77
:04F5F8002D8C2B8D9E
:01F5FC002CE2
:05F5FD00852D25E4B599
:04F602002502801F3E
:09F606007401B5253475328075DC
:06F60F0033D2753487754B
:06F6150035167536407544
:06F61B00377A7538AB756B
:04F62100391C8032DE
:07F625007532407533B87522
:06F62C0034BF75351075B6
:06F63200364075376C75CF
:07F6380038847539158018B4
:07F63F007532407533D575EB
:06F6460034A475352C759B
:06F64C0036807537F475ED
:05F6520038567539393E
:04F65700852B088572
:03F65B002C097502
:0AF65E000A00750B0090424075F0A1
:0EF668000FE412FA16AE82AF83A8F0F98E02FC
:09F676008F0388048905752942FF
:08F67F00C3E5369AE5379BE56F
:0AF68700389CE5399D4047747C254E
:05F6910029404185291C
:0CF696002A8A828B838CF0EDC002C00336
:0DF6A200C004C005C006C007C000C00112B2
:0EF6AF00F198D001D000D007D006D005D004CD
:0AF6BD00D003D002E52E2AFAE52F53
:0AF6C7003BFBE5303CFCE5313DFD66
:04F6D100052980AADD
:0AF6D500EEC3952EFAEF952FFBE827
:08F6DF009530FCE99531FD7541
:02F6E7002842B7
:09F6E900C3EA9532EB9533EC9570
:07F6F20034ED95354036E5CB
:06F6F9002860321528858F
:0AF6FF00282A8A828B838CF0EDC06C
:0EF7090002C003C004C00512F198D005D00460
:0BF71700D003D002EAC3952EFAEB9558
:08F722002FFBEC9530FCED9586
:04F72A0031FD80BB72
:04F72E00852B218581
:03F732002C22C2C4
:05F7350000852B828518
:03F73A002C8322FB
:0CF73D00E58275F008A4FAABF0EA2400A5
:0CF74900F582EB3400F583E090DF09F05E
:0AF75500EA2400FAEB3400FB8A827C
:0EF75F008B83A3E090DF0AF08A828B83A3A342
:0EF76D00E090DF0BF08A828B83A3A3A3E090D1
:0DF77B00DF1CF08A828B83A3A3A3A3E09080
:0EF78800DF1DF08A828B83A3A3A3A3A3E090CE
:04F79600DF1EF02260
:07F79A0085822612F0CC85E8
:06F7A10021828522830293
:02F7A700F23D31
:01F7A900223D
:07F7AA007521937522037520
:06F7B1002393752403758B
:06F7B7002502752600C2C8
:04F7BD0000C201C2C3
:05F7C100027527007530
:06F7C600280075298312E2
:08F7CC00F08B75820012F79A20
:02F7D400AA2861
:09F7D600C3EA9529400302F8681A
:0EF7DF008A82C00212F73D75E10290000A1204
:0CF7ED00F064D0027401B526117B5E7C34
:01F7F900010E
:09F7FA008B058C061BBBFF011CF2
:04F80300ED4E70F363
:0AF80700EA75F008A42400FB740069
:0EF8110035F0FC74062BFDE43CFE90DF3AE07F
:0CF81F00FF6307808D828E83EFF03000C5
:0EF82B002A74072BFFE43CF88D828E83E0F9EF
:0CF839008F828883E0F546C39950088D4B
:07F84500828E83E0FD8002CA
:02F84C00AD46C7
:08F84E008F828883EDF0800B2E
:0BF8560074072BF582E43CF583E4F01E
:07F8610075E1040A02F7D66D
:06F8680012F7A9E521B52D
:05F86E002308E522B5AE
:05F87300240302F7D49C
:07F878008523828524831221
:07F87F00F23D858223858321
:04F886002402F7D48D
:05F88A007A10E4FBFC14
:0EF88F00E58225E0F582E58333F583EB33FB5C
:0AF89D00EC33FCEB9508F5F0EC9558
:09F8A700094006FCABF0438201AC
:03F8B000DADD227C
:06F8B30012F956BC00032F
:03F8B90002FAA5AB
:08F8BC00EF60FA30D502B2D171
:08F8C400E583B4FF0302FABB67
:08F8CC00E582B4FF0302FABB60
:0BF8D400258340072482400B02FAA5A8
:08F8DF00248314500302FABB5C
:0EF8E700F582EA8DF0A4A8F0EA8EF0A428F8CD
:0EF8F500E435F0F9EB8DF0A428E935F0F9E4E4
:0EF9030033CA8FF0A429F9EA35F0FAEBF88E3A
:0EF91100F0A429F9EA35F0FAE433FBEC8DF0AE
:0EF91F00A429F9EA35F0FAE43BFBE88FF0A4E6
:0EF92D002AFAEB35F0FBE433CCFD8EF0A42A71
:0EF93B00FAEB35F0FBE43CFCED8FF0A42BFB67
:0AF94900EC35F0FC20E70312F9840E
:03F9530002FA8431
:0DF95600AA82AB83A2F73392D16002D2F7F0
:0EF96300F582ACF0E58124F9F8E6FD08E6FE39
:0EF971000886F008E6A2F73392D56002D2F7BE
:05F97F00F583AFF0224A
:06F03700E478FFF6D8FDAD
:02F98400780405
:0EF98600EC700DC9CACBFCE58224F8F582D8DE
:02F99400F1225E
:02F996007820D7
:0EF9980020E7111582C3E933F9EA33FAEB33A5
:06F9A600FBEC33FCD8EC81
:01F9AC002238
:08F015007900E94400601B7A58
:05F01D000090FB527899
:03F02200207593C3
:0AF0250004E493F2A308B80002050A
:08F02F0093D9F4DAF27593FFA6
:09F9AD00FCABF0AA83A982749E50
:02F9B600C2D1BC
:08F9B800F58212F98402FA84C1
:02F9C0007F9E28
:09F9C20012F9E730D10302FAA5A5
:0EF9CB00C3EF9582500974FFF5F0F583F582C5
:01F9D900220B
:05F9DA00790012FB0B97
:08F9DF0089828A838BF0EC227F
:0DF9E700AA82AB83A2F73392D16002D2F75F
:05F9F400F582ACF022D9
:0BF9F900E5828508F0A4C582C0F085FF
:0AFA040009F0A4D0F025F0C58385B9
:08FA0E0008F0A42583F5832212
:0CFA1600AAF0FBE5828508F0A4FCADF02E
:0CFA2200E5838508F0A42DFDE435F0FE1E
:0CFA2E00E5828509F0A42DFDE5F03EFE08
:0CFA3A00E433FFEA8508F0A42EFEE5F09E
:0CFA46003FFFE5838509F0A42EFEE5F0EB
:0CFA52003FFFE582850AF0A42EFEE5F0DF
:0BFA5E003FFFEB8508F0A42FFFEA85B6
:0AFA690009F0A42FFFE583850AF0E1
:0CFA7300A42FFFE582850BF0A42F8EF07D
:05FA7F008D838C822242
:08F03D007800E84400600A7944
:03F04500007593C0
:06F0480000E4F309D8FC0E
:08F04E007820E84404600C790D
:0BF0560005900000E4F0A3D8FCD9FAFC
:06FA8400B98003EA13B390
:0EFA8A004010EA2401FAE43BFBE43CFC50048B
:04FA98007C800582E7
:09FA9C00BC000EBB000BBA00080F
:08FAA500E4F5F0F583F582227F
:0EFAAD00A2D1E582138CF092F78B838A82221D
:0DFABB00E4F583F58275F080F4A2D11322EA
:0BFAC800E4F583F58275F0C0747F2226
:03F00800758146C9
:0AF00B0012FB4EE582600302F003E1
:0EFAD300C2D5E58330E70DD2D5E4C39582F5A8
:06FAE10082E49583F58329
:0AFAE700E50930E70DB2D5E4C39540
:05FAF10008F508E49592
:03FAF60009F50906
:0EFAF90012F88A30D50BE4C39582F582E495AD
:03FB070083F58300
:01FB0A0022D8
:09FB0B006040F82582500274FFED
:0EFB1400F582E824F8501ECCCBCAF9E4CC24CC
:0EFB2200F85014CBCAF9E4CB24F8500BCAF902
:09FB3000E4CA24F8500379002214
:05FB390024086010F833
:0EFB3E00C3EC13FCEB13FBEA13FAE913F9D83E
:01FB4C00F1C7
:01FB4D002295
:04FB4E00758200229A
:00000001FF
